:020000040000FA
:0408000085EF09F087
:1008100003B28CEF05F0F2B4AAEF05F09EB0B2EF90
:1008200005F09EB2BAEF05F0F2A81AEF04F0F2B2AA
:100830003AEF04F09EB61FEF04F034EF09F09E96F5
:1008400000011750000A0AE000011750010A0AE0EF
:1008500000011750020A0AE034EF09F086EC24F098
:1008600034EF09F07EEC26F034EF09F060EC27F06D
:1008700034EF09F0CD90F2929EA044EF04F0010114
:10088000533F44EF04F0542BB2C1B6F1B3C1B7F1FA
:10089000B4C1B8F1B5C1B9F1AEC1B2F1AFC1B3F1F4
:1008A000B0C1B4F1B1C1B5F1AAC1AEF1ABC1AFF104
:1008B000ACC1B0F1ADC1B1F1A6C1AAF1A7C1ABF114
:1008C000A8C1ACF1A9C1ADF1A2C1A6F1A3C1A7F124
:1008D000A4C1A8F1A5C1A9F19EC1A2F19FC1A3F134
:1008E000A0C1A4F1A1C1A5F19AC19EF19BC19FF144
:1008F0009CC1A0F19DC1A1F1CECF9AF1CFCF9BF1C8
:1009000053C19CF154C19DF1CF6ACE6A0101536B72
:10091000546B9E90CD800FBC0F8E0FBA93EF04F0F6
:100920000F8A34EF09F013880F8C0FBED0EF04F05C
:100930009AC19EF19BC19FF19CC1A0F19DC1A1F103
:100940009EC1A2F19FC1A3F1A0C1A4F1A1C1A5F1D3
:10095000A2C1A6F1A3C1A7F1A4C1A8F1A5C1A9F1A3
:10096000A6C1AAF1A7C1ABF1A8C1ACF1A9C1ADF173
:10097000AAC1AEF1ABC1AFF1ACC1B0F1ADC1B1F143
:10098000AEC1B2F1AFC1B3F1B0C1B4F1B1C1B5F113
:10099000B2C1B6F1B3C1B7F1B4C1B8F1B5C1B9F1E3
:1009A00001015E6B5F6B606B616B9A515E279B51BF
:1009B0005F239C5160239D5161239E515E279F516F
:1009C0005F23A0516023A1516123A2515E27A3514F
:1009D0005F23A4516023A5516123A6515E27A7512F
:1009E0005F23A8516023A9516123AA515E27AB510F
:1009F0005F23AC516023AD516123AE515E27AF51EF
:100A00005F23B0516023B1516123B2515E27B351CE
:100A10005F23B4516023B5516123B6515E27B751AE
:100A20005F23B8516023B9516123D890010161332C
:100A300060335F335E33D8900101613360335F33DD
:100A40005E33D8900101613360335F335E3300C1A0
:100A50000CF101C10DF102C10EF103C10FF104C18E
:100A600010F105C111F106C112F107C113F108C15E
:100A700014F109C115F10AC116F10BC117F134C106
:100A800035F111B84FEF05F00101620E046F010E50
:100A9000056F000E066F000E076F58EF05F001019D
:100AA000A70E046F020E056F000E066F000E076F93
:100AB0005EC100F15FC101F160C102F161C103F1EA
:100AC000EAEC22F003BF04D01CBE02D01CA0108CA4
:100AD00011A070EF05F010BA70EF05F00F80108ACA
:100AE0000CC100F10DC101F10EC102F10FC103F102
:100AF00010C104F111C105F112C106F113C107F1D2
:100B000014C108F115C109F116C10AF117C10BF1A1
:100B100035C134F134EF09F00392ABB2AB98AB8836
:100B2000030103EE00F080517F0BE92604C0EFFFC4
:100B3000802B8151805D700BD8A48B820000805186
:100B4000815D700BD8A48B9281518019D8B4079025
:100B500034EF09F0F2940101453F34EF09F0462BE0
:100B600034EF09F09E900101533F34EF09F0542B0C
:100B700034EF09F09E9211B830EF07F08BB4C8EF54
:100B800005F010ACC8EF05F08B84109CC9EF05F0A0
:100B90008B94C3CF55F1C4CF56F1C28207B438EF5E
:100BA00006F047C14BF148C14CF149C14DF14AC172
:100BB0004EF15EC162F15FC163F160C164F161C178
:100BC00065F113A8E6EF05F0138C13989AC1BAF1FA
:100BD0009BC1BBF19CC1BCF19DC1BDF19EC1BEF1E9
:100BE0009FC1BFF1A0C1C0F1A1C1C1F1A2C1C2F1B9
:100BF000A3C1C3F1A4C1C4F1A5C1C5F1A6C1C6F189
:100C0000A7C1C7F1A8C1C8F1A9C1C9F1AAC1CAF158
:100C1000ABC1CBF1ACC1CCF1ADC1CDF1AEC1CEF128
:100C2000AFC1CFF1B0C1D0F1B1C1D1F1B2C1D2F1F8
:100C3000B3C1D3F1B4C1D4F1B5C1D5F1B6C1D6F1C8
:100C4000B7C1D7F1B8C1D8F1B9C1D9F10101555136
:100C50005B2756515C23E86A5D230E2E38EF06F0C1
:100C60005CC157F15DC158F15B6B5C6B5D6B078ECE
:100C70000201002F34EF09F03C0E006F1D50E00B15
:100C8000E00AE86612881BBE02D01BB4108E00C1B9
:100C90000CF101C10DF102C10EF103C10FF104C14C
:100CA00010F105C111F106C112F107C113F108C11C
:100CB00014F109C115F10AC116F10BC117F134C1C4
:100CC00035F101018E676CEF06F08F676CEF06F06F
:100CD00090676CEF06F0916770EF06F0A1EF06F0F9
:100CE00092C100F193C101F194C102F195C103F1E8
:100CF0000101010E046F000E056F000E066F000E5D
:100D0000076FEAEC22F000C192F101C193F102C138
:100D100094F103C195F10101006796EF06F00167B8
:100D200096EF06F0026796EF06F00367A1EF06F074
:100D30008EC192F18FC193F190C194F191C195F15F
:100D40000F80D57ED5BE6ED0D6CF47F1D7CF48F134
:100D500045C149F1E86AE8CF4AF1138A1CBE02D0C6
:100D60001CA0108C109047C100F148C101F149C18D
:100D700002F14AC103F101010A0E046F000E056F72
:100D8000000E066F000E076FEAEC22F003AF108032
:100D9000010154A7D8EF06F00F9A0F9C0F9E010196
:100DA000000E5E6F600E5F6F3D0E606F080E616F2C
:100DB000010147BFE8EF06F04867E8EF06F0496732
:100DC000E8EF06F04A67E8EF06F0F2880DEF07F06B
:100DD000F2985E6B5F6B606B616B9A6B9B6B9C6B4D
:100DE0009D6B9E6B9F6BA06BA16BA26BA36BA46BA7
:100DF000A56BA66BA76BA86BA96BAA6BAB6BAC6B57
:100E0000AD6BAE6BAF6BB06BB16BB26BB36BB46B06
:100E1000B56BB66BB76BB86BB96BD76AD66A0101A5
:100E2000456B466B0CC100F10DC101F10EC102F121
:100E30000FC103F110C104F111C105F112C106F196
:100E400013C107F114C108F115C109F116C10AF166
:100E500017C10BF135C134F134EF09F034EF09F06B
:100E60000201002F8BEF08F0D59ED6CF47F1D7CFE8
:100E700048F145C149F1E86AE8CF4AF1138AD76AD7
:100E8000D66A0101456B466BD58E1D50E00BE00A1A
:100E9000E86612881BBE02D01BB4108E1AAE1F8CDF
:100EA00000C10CF101C10DF102C10EF103C10FF13E
:100EB00004C110F105C111F106C112F107C113F10E
:100EC00008C114F109C115F10AC116F10BC117F1DE
:100ED00034C135F10FA0109A11B87AEF07F0010173
:100EE000620E046F010E056F000E066F000E076F95
:100EF00083EF07F00101A70E046F020E056F000ECD
:100F0000066F000E076F47C100F148C101F149C1EA
:100F100002F14AC103F1EAEC22F003BF96EF07F0B9
:100F20001CBE02D01CA0108C11B00F800CC100F1AF
:100F30000DC101F10EC102F10FC103F110C104F1A5
:100F400011C105F112C106F113C107F114C108F175
:100F500015C109F116C10AF117C10BF135C134F100
:100F600002013C0E006F00C10CF101C10DF102C184
:100F70000EF103C10FF104C110F105C111F106C159
:100F800012F107C113F108C114F109C115F10AC129
:100F900016F10BC117F134C135F101018E67D8EF9D
:100FA00007F08F67D8EF07F09067D8EF07F09167E9
:100FB000DCEF07F00DEF08F092C100F193C101F1F1
:100FC00094C102F195C103F10101010E046F000EFD
:100FD000056F000E066F000E076FEAEC22F000C1ED
:100FE00092F101C193F102C194F103C195F10101A4
:100FF000006702EF08F0016702EF08F0026702EFF6
:1010000008F003670DEF08F08EC192F18FC193F1E4
:1010100090C194F191C195F10F80109047C100F1FA
:1010200048C101F149C102F14AC103F101010A0EAF
:10103000046F000E056F000E066F000E076FEAECDE
:1010400022F003AF1080010154A733EF08F00F9A8C
:101050000F9C0F9E0101000E5E6F600E5F6F3D0ED4
:10106000606F080E616F47C100F148C101F149C1CD
:1010700002F14AC103F10101140E046F050E056F60
:10108000000E066F000E076FEAEC22F003AF4CEF84
:1010900008F0F28871EF08F0F2985E6B5F6B606B9E
:1010A000616B9A6B9B6B9C6B9D6B9E6B9F6BA06B3C
:1010B000A16BA26BA36BA46BA56BA66BA76BA86BB4
:1010C000A96BAA6BAB6BAC6BAD6BAE6BAF6BB06B64
:1010D000B16BB26BB36BB46BB56BB66BB76BB86B14
:1010E000B96B0CC100F10DC101F10EC102F10FC1CC
:1010F00003F110C104F111C105F112C106F113C1D0
:1011000007F114C108F115C109F116C10AF117C19F
:101110000BF135C134F13DEC27F0206629D01FAE2C
:1011200011D01F9E208E1BAE07D0176A040E186EBA
:10113000196A86EC24F01CD0176A186A196A86ECC2
:1011400024F016D01FAC09D01F9C208C010E176E06
:10115000186A196A7EEC26F00BD01FAA09D01F9AD4
:10116000208A020E176E186A196A60EC27F000D008
:101170008BB4C2EF08F010ACC2EF08F08B84109C67
:10118000C3EF08F08B94C3CF55F1C4CF56F1C282A0
:1011900007B432EF09F047C14BF148C14CF149C1E6
:1011A0004DF14AC14EF15EC162F15FC163F160C1B0
:1011B00064F161C165F113A8E0EF08F0138C139896
:1011C0009AC1BAF19BC1BBF19CC1BCF19DC1BDF1FB
:1011D0009EC1BEF19FC1BFF1A0C1C0F1A1C1C1F1CB
:1011E000A2C1C2F1A3C1C3F1A4C1C4F1A5C1C5F19B
:1011F000A6C1C6F1A7C1C7F1A8C1C8F1A9C1C9F16B
:10120000AAC1CAF1ABC1CBF1ACC1CCF1ADC1CDF13A
:10121000AEC1CEF1AFC1CFF1B0C1D0F1B1C1D1F10A
:10122000B2C1D2F1B3C1D3F1B4C1D4F1B5C1D5F1DA
:10123000B6C1D6F1B7C1D7F1B8C1D8F1B9C1D9F1AA
:10124000010155515B2756515C23E86A5D230E2E40
:1012500032EF09F05CC157F15DC158F15B6B5C6B1B
:101260005D6B078E34EF09F002C0E0FF005001C053
:10127000D8FF1000A6B23AEF09F00CC0A9FF0BC0CE
:10128000A8FFA69EA69CA684F29E550EA76EAA0E47
:10129000A76EA682F28EA694A6B24CEF09F00C2A95
:1012A0001200A96EA69EA69CA680A8500C2A120029
:1012B00004012C0E826F6EEC0BF0FFEC23F00C504F
:1012C00051EC09F0E8CF00F10C5051EC09F0E8CFF7
:1012D00001F101AF71EF09F00101FF0E026FFF0E86
:1012E000036F88EC23F029677DEF09F00401200EDD
:1012F000826F6EEC0BF082EF09F004012D0E826F0D
:101300006EEC0BF092EC21F0120015941596076A22
:101310000F6A106A116A126A136A166A0F010E0EBA
:10132000C16E860EC06E030EC26E0F01896A110E69
:10133000926E080E8A6EF10E936E8B6A980E946E02
:10134000F18EFC0E51EC09F0E8CF0BF00BA01180F0
:101350000BA211820BA411840BA81188C90E51ECA9
:1013600009F0E8CF1AF0CA0E51EC09F0E8CF1BF0F3
:10137000CB0E51EC09F0E8CF1CF0CC0E51EC09F08B
:10138000E8CF1DF0FB0E51EC09F0E8CF38F0CE0E9F
:1013900051EC09F0E8CF14F0CD0E51EC09F0E8CF94
:1013A00037F01F6A206A0E6A01015B6B5C6B5D6B34
:1013B000576B586BF29A0101476B486B496B4A6B4C
:1013C0004B6B4C6B4D6B4E6B4F6B506B516B526B51
:1013D000456B466BD76AD66A0F01280ED56EF28A26
:1013E0009D90B00ECD6E01015E6B5F6B606B616BAB
:1013F000626B636B646B656B666B676B686B696B69
:10140000536B546BCF6ACE6A0F9A0F9C0F9E9D80D0
:10141000760ECA6E9D8202013C0E006FCC6A160EDB
:1014200051EC09F0E8CF00F1170E51EC09F0E8CFCC
:1014300001F1180E51EC09F0E8CF02F1190E51EC50
:1014400009F0E8CF03F1010103AF41EF0AF0FFEC2F
:1014500023F0160E0C6E00C10BF03AEC09F0170EDB
:101460000C6E01C10BF03AEC09F0180E0C6E02C1C3
:101470000BF03AEC09F0190E0C6E03C10BF03AECCC
:1014800009F000C18EF101C18FF102C190F103C1D9
:1014900091F100C192F101C193F102C194F103C134
:1014A00095F11A0E51EC09F0E8CF00F11B0E51EC4A
:1014B00009F0E8CF01F11C0E51EC09F0E8CF02F180
:1014C0001D0E51EC09F0E8CF03F1010103AF97EFD6
:1014D0000AF0FFEC23F01A0E0C6E00C10BF03AEC90
:1014E00009F01B0E0C6E01C10BF03AEC09F01C0E5A
:1014F0000C6E02C10BF03AEC09F01D0E0C6E03C12C
:101500000BF03AEC09F01A0E51EC09F0E8CF00F1BB
:101510001B0E51EC09F0E8CF01F11C0E51EC09F063
:10152000E8CF02F11D0E51EC09F0E8CF03F100C144
:1015300096F101C197F102C198F103C199F1240E0E
:10154000AC6E900EAB6E240EAC6E080EB86E000E34
:10155000B06E1F0EAF6E0401806B816B0F01900E99
:10156000AB6E0F019D8A0301806B816BC26B8B9206
:10157000176A186A196A9D8607900001F28EF28C2C
:1015800007B03BEF20F00FB02BEF19F010BE2BEFA0
:1015900019F012B82BEF19F00301805181197F0B5C
:1015A000D8B43BEF20F013EE00F081517F0BE12621
:1015B000812BE7CFE8FFE00BD8B43BEF20F023EE20
:1015C00082F0C2513F0BD926E7CFDFFFC22BDF509D
:1015D000780AD8A43BEF20F0078092C100F193C1B4
:1015E00001F194C102F195C103F10101040E046FF0
:1015F000000E056F000E066F000E076FEAEC22F07A
:1016000000AF0CEF0BF00101030E926F000E936F11
:10161000000E946F000E956F03018251720AD8B4C8
:10162000ACEF18F08251520AD8B4ACEF18F08251E6
:10163000750AD8B4ACEF18F08251680AD8B482EFBA
:101640000BF08251630AD8B4F5EF1CF08251690A9D
:10165000D8B471EF13F082517A0AD8B484EF14F041
:101660008251490AD8B410EF13F08251500AD8B40D
:101670001AEF12F08251700AD8B462EF12F0825160
:10168000540AD8B492EF12F08251740AD8B4DDEF44
:1016900012F08251410AD8B4FDEF0CF082514B0A8E
:1016A000D8B4FAEF0BF082516D0AD8B46DEF11F097
:1016B00082514D0AD8B486EF11F08251730AD8B422
:1016C000DCEF17F08251530AD8B441EF18F0825181
:1016D000590AD8B4BEEF10F02CEF1DF0040114EE3F
:1016E00000F080517F0BE12682C4E7FF802B1200BF
:1016F00004010D0E826F6EEC0BF00A0E826F6EEC21
:101700000BF012000401680E826F6EEC0BF0040106
:101710002C0E826F6EEC0BF0FFEC23F033C000F167
:1017200034C001F1010188EC23F02EC182F40401E0
:10173000300E82276EEC0BF02FC182F40401300EC4
:1017400082276EEC0BF030C182F40401300E822748
:101750006EEC0BF031C182F40401300E82276EEC86
:101760000BF032C182F40401300E82276EEC0BF0D4
:1017700033C182F40401300E82276EEC0BF00401B9
:101780002C0E826F6EEC0BF0FFEC23F035C000F1F5
:1017900036C001F188EC23F02EC182F40401300E32
:1017A00082276EEC0BF02FC182F40401300E8227E9
:1017B0006EEC0BF030C182F40401300E82276EEC27
:1017C0000BF031C182F40401300E82276EEC0BF075
:1017D00032C182F40401300E82276EEC0BF033C16B
:1017E00082F40401300E82276EEC0BF060EC27F0DF
:1017F0002AEF1DF004014B0E826F6EEC0BF004011A
:101800002C0E826F6EEC0BF081B802D037B630D060
:1018100003018351430AD8B43FEF0CF00301835115
:10182000630AD8B441EF0CF003018351520AD8B4D3
:1018300043EF0CF003018351720AD8B445EF0CF06A
:1018400003018351470AD8B447EF0CF003018351D9
:10185000670AD8B449EF0CF003018351540AD8B495
:101860004BEF0CF003018351740AD8B4BBEF0CF0BA
:1018700003018351550AD8B44DEF0CF083D0378063
:101880007BD0379079D0378277D0379275D0378434
:1018900073D0379471D037866FD084C330F185C34D
:1018A00031F186C332F187C333F10101296B4DEC6D
:1018B00024F0C4EC23F000C104F101C105F102C120
:1018C00006F103C107F140EC24F0200EF86EF76A30
:1018D000F66A0900F5CF2CF10900F5CF2DF10900CA
:1018E000F5CF2EF10900F5CF2FF10900F5CF30F13A
:1018F0000900F5CF31F10900F5CF32F10900F5CF3C
:1019000033F10101296B4DEC24F0C4EC23F0EAEC37
:1019100022F00101006794EF0CF0016794EF0CF0E6
:10192000026794EF0CF0036701D025D004014E0E3E
:10193000826F6EEC0BF004016F0E826F6EEC0BF099
:1019400004014D0E826F6EEC0BF00401610E826F8C
:101950006EEC0BF00401740E826F6EEC0BF0040160
:10196000630E826F6EEC0BF00401680E826F6EECFA
:101970000BF02AEF1DF03796CD0E0C6E37C00BF032
:101980003AEC09F0CD0E51EC09F0E8CF37F037B062
:1019900006D00401630E826F6EEC0BF005D00401DB
:1019A000430E826F6EEC0BF037B206D00401720E5C
:1019B000826F6EEC0BF005D00401520E826F6EEC5C
:1019C0000BF037B406D00401670E826F6EEC0BF09B
:1019D00005D00401470E826F6EEC0BF037B606D0CF
:1019E0000401740E826F6EEC0BF005D00401540EEE
:1019F000826F6EEC0BF02AEF1DF00401410E826F36
:101A00006EEC0BF003018351310AD8B4DEEF0FF016
:101A100003018351320AD8B40EEF0FF00301835152
:101A2000330AD8B497EF0EF003018351340AD8B4C7
:101A300087EF0DF003018351350AD8B427EF0DF07D
:101A400004013F0E826F6EEC0BF02AEF1DF00301D4
:101A50008451300AD8B44DEF0DF003018451310A9E
:101A6000D8B450EF0DF003018451650AD8B441EFAA
:101A70000DF003018451640AD8B444EF0DF051EF26
:101A80000DF0389045EF0DF03880FB0E0C6E38C02D
:101A90000BF03AEC09F051EF0DF08B9051EF0DF097
:101AA0008B800401350E826F6EEC0BF004012C0E5E
:101AB000826F6EEC0BF08BB065EF0DF00401300E11
:101AC000826F6EEC0BF06AEF0DF00401310E826F45
:101AD0006EEC0BF004012C0E826F6EEC0BF0FB0E23
:101AE00051EC09F0E8CF38F038A07EEF0DF004019A
:101AF000640E826F6EEC0BF083EF0DF00401650E47
:101B0000826F6EEC0BF085EF0DF02AEF1DF0CC0E1E
:101B100051EC09F0E8CF0BF004012C0E826F6EEC53
:101B20000BF003018451310AD8B4ABEF0DF003017F
:101B30008451300AD8B4ADEF0DF0030184514D0A41
:101B4000D8B4B7EF0DF003018451540AD8B4BEEFF6
:101B50000DF0D5EF0DF08A8401D08A940BAE04D03D
:101B60000BAC02D00BBA21D0E00E0B1218D01F0E16
:101B70000B168539E844E00B0B1211D0E00E0B1662
:101B800040EC24F085C332F186C333F10101296BA7
:101B90004DEC24F0C4EC23F000511F0B0B12CC0EC3
:101BA0000C6E0BC00BF03AEC09F00401340E826F9E
:101BB0006EEC0BF004012C0E826F6EEC0BF0CC0E71
:101BC00051EC09F0E8CF1DF08AB406D00401300EC4
:101BD000826F6EEC0BF005D00401310E826F6EEC5B
:101BE0000BF004012C0E826F6EEC0BF01D38E840F8
:101BF000070BE8CF82F40401300E82276EEC0BF065
:101C000004012C0E826F6EEC0BF0FFEC23F01D50E4
:101C10001F0BE8CF00F188EC23F032C182F40401FD
:101C2000300E82276EEC0BF033C182F40401300ECB
:101C300082276EEC0BF004012C0E826F6EEC0BF021
:101C4000FFEC23F031C000F100AF0BD0FF0E016FAD
:101C5000FF0E026FFF0E036F04012D0E826F6EECFC
:101C60000BF088EC23F031C182F40401300E82279E
:101C70006EEC0BF032C182F40401300E82276EEC60
:101C80000BF033C182F40401300E82276EEC0BF0AE
:101C900004012C0E826F6EEC0BF0FFEC23F030C0D1
:101CA00000F188EC23F031C182F40401300E822768
:101CB0006EEC0BF032C182F40401300E82276EEC20
:101CC0000BF033C182F40401300E82276EEC0BF06E
:101CD00004012C0E826F6EEC0BF0FFEC23F032C08F
:101CE00000F100AF0BD0FF0E016FFF0E026FFF0E71
:101CF000036F04012D0E826F6EEC0BF088EC23F065
:101D000031C182F40401300E82276EEC0BF032C137
:101D100082F40401300E82276EEC0BF033C182F4A2
:101D20000401300E82276EEC0BF02AEF1DF0CB0E73
:101D300051EC09F0E8CF0BF004012C0E826F6EEC31
:101D40000BF003018451450AD8B4BBEF0EF0030138
:101D50008451440AD8B4BEEF0EF003018451300A16
:101D6000D8B4C1EF0EF003018451310AD8B4C5EFE5
:101D70000EF0D0EF0EF00B9ECAEF0EF00B8ECAEFF6
:101D80000EF0FC0E0B16CAEF0EF0FC0E0B160B80BD
:101D9000CAEF0EF0CB0E0C6E0BC00BF03AEC09F054
:101DA0000401330E826F6EEC0BF004012C0E826F77
:101DB0006EEC0BF0CB0E51EC09F0E8CF1CF01CBE22
:101DC000E9EF0EF00401450E826F6EEC0BF0EEEFC2
:101DD0000EF00401440E826F6EEC0BF004012C0E29
:101DE000826F6EEC0BF00401300E826F6EEC0BF024
:101DF00004012C0E826F6EEC0BF01CB007EF0FF09D
:101E00000401300E826F6EEC0BF00CEF0FF004014A
:101E1000310E826F6EEC0BF02AEF1DF0CA0E51EC02
:101E200009F0E8CF0BF004012C0E826F6EEC0BF082
:101E300003018451450AD8B44AEF0FF003018451DD
:101E4000440AD8B44DEF0FF0030184514D0AD8B4C1
:101E500056EF0FF003018451410AD8B450EF0FF050
:101E600003018451460AD8B453EF0FF003018451A3
:101E7000560AD8B45EEF0FF003018451500AD8B46B
:101E800069EF0FF003018451520AD8B46CEF0FF0E0
:101E900075EF0FF00B9E6FEF0FF00B8E6FEF0FF0E3
:101EA0000B9C6FEF0FF00B8C6FEF0FF0FC0E0B160F
:101EB00085C3E8FF030B0B126FEF0FF0C70E0B1675
:101EC00085C3E8FF070BE846E846E8460B126FEFCC
:101ED0000FF00B846FEF0FF00B946FEF0FF0CA0E43
:101EE0000C6E0BC00BF03AEC09F0CA0E51EC09F085
:101EF000E8CF1BF00401320E826F6EEC0BF0040190
:101F00002C0E826F6EEC0BF01BBE8EEF0FF00401F7
:101F1000450E826F6EEC0BF093EF0FF00401440E50
:101F2000826F6EEC0BF004012C0E826F6EEC0BF0E6
:101F30001BC0E8FF030BE8CF82F40401300E8227B8
:101F40006EEC0BF004012C0E826F6EEC0BF01BBCE0
:101F5000B1EF0FF00401410E826F6EEC0BF0B6EFA3
:101F60000FF00401460E826F6EEC0BF004012C0E94
:101F7000826F6EEC0BF01BC0E8FF380BE842E842C2
:101F8000E842E8CF82F40401300E82276EEC0BF0B9
:101F900004012C0E826F6EEC0BF01BB4D7EF0FF028
:101FA0000401520E826F6EEC0BF0DCEF0FF00401B7
:101FB000500E826F6EEC0BF02AEF1DF0C90E51EC43
:101FC00009F0E8CF0BF004012C0E826F6EEC0BF0E1
:101FD00003018451450AD8B4FCEF0FF0030184518A
:101FE000440AD8B4FFEF0FF0030184514D0AD8B46E
:101FF00002EF10F010EF10F00B9E0AEF10F00B8EB6
:102000000AEF10F0F80E0B1685C3E8FF070B0B1252
:102010000AEF10F0C90E0C6E0BC00BF03AEC09F091
:102020000401310E826F6EEC0BF004012C0E826FF6
:102030006EEC0BF0C90E51EC09F0E8CF1AF01ABEA5
:1020400006D00401450E826F6EEC0BF005D0040142
:10205000440E826F6EEC0BF004012C0E826F6EEC5E
:102060000BF01AC0E8FF070BE8CF82F40401300E32
:1020700082276EEC0BF004012C0E826F6EEC0BF0DD
:102080000780FFEC23F02CC0E8FF003B0043004337
:10209000030B88EC23F033C182F40401300E822755
:1020A0006EEC0BF004012C0E826F6EEC0BF0FFEC6B
:1020B00023F02CC001F1019F019D2DC000F1010111
:1020C00088EC23F02FC182F40401300E82276EECDD
:1020D0000BF030C182F40401300E82276EEC0BF05D
:1020E00031C182F40401300E82276EEC0BF032C154
:1020F00082F40401300E82276EEC0BF033C182F4BF
:102100000401300E82276EEC0BF004012C0E826F5E
:102110006EEC0BF0FFEC23F02EC001F12FC000F1AC
:10212000D89001330033D89001330033010188EC9B
:1021300023F02FC182F40401300E82276EEC0BF0E5
:1021400030C182F40401300E82276EEC0BF031C1F5
:1021500082F40401300E82276EEC0BF032C182F45F
:102160000401300E82276EEC0BF033C182F40401BF
:10217000300E82276EEC0BF02AEF1DF0FC0E51ECB6
:1021800009F0E8CF0BF003018351520AD8B4F5EF00
:1021900010F003018351720AD8B4F8EF10F0030174
:1021A0008351500AD8B4FBEF10F003018351700A39
:1021B000D8B4FEEF10F003018351550AD8B401EFF3
:1021C00011F003018351750AD8B404EF11F0030133
:1021D0008351430AD8B40DEF11F003018351630A10
:1021E000D8B410EF11F019EF11F00B9013EF11F0BC
:1021F0000B8013EF11F00B9213EF11F00B8213EF22
:1022000011F00B9413EF11F00B8413EF11F00B96F8
:1022100013EF11F00B8613EF11F00B9813EF11F081
:102220000B8813EF11F0FC0E0C6E0BC00BF03AECA8
:1022300009F00401590E826F6EEC0BF011901192AF
:1022400011941198FC0E51EC09F0E8CF0BF00BA0A3
:1022500011800BA211820BA411840BA8118811A06C
:1022600039EF11F00401520E826F6EEC0BF03EEF6D
:1022700011F00401720E826F6EEC0BF011A848EFA2
:1022800011F00401430E826F6EEC0BF04DEF11F074
:102290000401630E826F6EEC0BF011A257EF11F088
:1022A0000401500E826F6EEC0BF05CEF11F0040134
:1022B000700E826F6EEC0BF011A466EF11F004014A
:1022C000550E826F6EEC0BF06BEF11F00401750E82
:1022D000826F6EEC0BF02AEF1DF004016D0E826F21
:1022E0006EEC0BF003018351300AD8B4CAEF11F041
:1022F00003018351310AD8B4DDEF11F0030183519A
:10230000320AD8B4F0EF11F02CEF1DF081B803D0F1
:1023100037B42AEF1DF004014D0E826F6EEC0BF006
:1023200040EC24F084C331F185C332F186C333F12C
:102330000101296B4DEC24F0C4EC23F0030183511F
:10234000300AD8B4B2EF11F003018351310AD8B486
:10235000BAEF11F003018351320AD8B4C2EF11F081
:102360002CEF1DF0FD0E0C6E00C10BF03AEC09F0E5
:10237000CAEF11F0FE0E0C6E00C10BF03AEC09F042
:10238000DDEF11F0FF0E0C6E00C10BF03AEC09F01E
:10239000F0EF11F00401300E826F6EEC0BF00401CF
:1023A0002C0E826F6EEC0BF0FFEC23F0FD0E51EC67
:1023B00009F0E8CF00F101EF12F00401310E826F55
:1023C0006EEC0BF004012C0E826F6EEC0BF0FFEC48
:1023D00023F0FE0E51EC09F0E8CF00F101EF12F00E
:1023E0000401320E826F6EEC0BF0FFEC23F004015F
:1023F0002C0E826F6EEC0BF0FF0E51EC09F0E8CF63
:1024000000F188EC23F031C182F40401300E822700
:102410006EEC0BF032C182F40401300E82276EECB8
:102420000BF033C182F40401300E82276EEC0BF006
:102430002AEF1DF081B803D037B210EF13F083C339
:102440002AF184C32BF185C32CF186C32DF187C3F8
:102450002EF188C32FF189C330F18AC331F18BC3C8
:1024600032F18CC333F101014DEC24F0C4EC23F0C4
:10247000160E0C6E00C10BF03AEC09F0170E0C6E44
:1024800001C10BF03AEC09F0180E0C6E02C10BF012
:102490003AEC09F0190E0C6E03C10BF03AEC09F09E
:1024A00000C18EF101C18FF102C190F103C191F120
:1024B00000C192F101C193F102C194F103C195F100
:1024C00010EF13F081B803D037B210EF13F083C3CD
:1024D0002AF184C32BF185C32CF186C32DF187C368
:1024E0002EF188C32FF189C330F18AC331F18BC338
:1024F00032F18CC333F101014DEC24F0C4EC23F034
:1025000000C18EF101C18FF102C190F103C191F1BF
:1025100000C192F101C193F102C194F103C195F19F
:1025200010EF13F081B803D037B210EF13F083C36C
:102530002AF184C32BF185C32CF186C32DF187C307
:102540002EF188C32FF189C330F18AC331F18CC3D6
:1025500032F18DC333F101014DEC24F0C4EC23F0D2
:102560000101000E046F000E056F010E066F000ED4
:10257000076FFBEC22F01A0E0C6E00C10BF03AEC68
:1025800009F01B0E0C6E01C10BF03AEC09F01C0EA9
:102590000C6E02C10BF03AEC09F01D0E0C6E03C17B
:1025A0000BF03AEC09F000C196F101C197F102C1BC
:1025B00098F103C199F110EF13F081B803D037B24D
:1025C00010EF13F083C32AF184C32BF185C32CF1E0
:1025D00086C32DF187C32EF188C32FF189C330F153
:1025E0008AC331F18CC332F18DC333F101014DEC5B
:1025F00024F0C4EC23F00101000E046F000E056FFF
:10260000010E066F000E076FFBEC22F000C196F181
:1026100001C197F102C198F103C199F110EF13F0D4
:10262000160E51EC09F0E8CF00F1170E51EC09F04D
:10263000E8CF01F1180E51EC09F0E8CF02F1190EC4
:1026400051EC09F0E8CF03F188EC23F04BEC21F0DA
:102650000401730E826F6EEC0BF004012C0E826F7E
:102660006EEC0BF08EC100F18FC101F190C102F14F
:1026700091C103F188EC23F04BEC21F00401730EBF
:10268000826F6EEC0BF004012C0E826F6EEC0BF07F
:102690001A0E51EC09F0E8CF00F11B0E51EC09F0D5
:1026A000E8CF01F11C0E51EC09F0E8CF02F11D0E4C
:1026B00051EC09F0E8CF03F147EC1DF004012C0EBA
:1026C000826F6EEC0BF096C100F197C101F198C1D9
:1026D00002F199C103F147EC1DF078EC0BF02CEFFF
:1026E0001DF00401690E826F6EEC0BF004012C0EDC
:1026F000826F6EEC0BF00101040E006F000E016F93
:10270000000E026F000E036F88EC23F02CC182F4E0
:102710000401300E82276EEC0BF02DC182F404010F
:10272000300E82276EEC0BF02EC182F40401300EC5
:1027300082276EEC0BF02FC182F40401300E822749
:102740006EEC0BF030C182F40401300E82276EEC87
:102750000BF031C182F40401300E82276EEC0BF0D5
:1027600032C182F40401300E82276EEC0BF033C1CB
:1027700082F40401300E82276EEC0BF004012C0E63
:10278000826F6EEC0BF00101030E006F000E016F03
:10279000000E026F000E036F88EC23F02CC182F450
:1027A0000401300E82276EEC0BF02DC182F404017F
:1027B000300E82276EEC0BF02EC182F40401300E35
:1027C00082276EEC0BF02FC182F40401300E8227B9
:1027D0006EEC0BF030C182F40401300E82276EECF7
:1027E0000BF031C182F40401300E82276EEC0BF045
:1027F00032C182F40401300E82276EEC0BF033C13B
:1028000082F40401300E82276EEC0BF004012C0ED2
:10281000826F6EEC0BF00101520E006F000E016F23
:10282000000E026F000E036F88EC23F02CC182F4BF
:102830000401300E82276EEC0BF02DC182F40401EE
:10284000300E82276EEC0BF02EC182F40401300EA4
:1028500082276EEC0BF02FC182F40401300E822728
:102860006EEC0BF030C182F40401300E82276EEC66
:102870000BF031C182F40401300E82276EEC0BF0B4
:1028800032C182F40401300E82276EEC0BF033C1AA
:1028900082F40401300E82276EEC0BF004012C0E42
:1028A000826F6EEC0BF0200EF86EF76AF66A040188
:1028B0000900F5CF82F46EEC0BF00900F5CF82F43D
:1028C0006EEC0BF00900F5CF82F46EEC0BF0090012
:1028D000F5CF82F46EEC0BF00900F5CF82F46EECCC
:1028E0000BF00900F5CF82F46EEC0BF00900F5CF88
:1028F00082F46EEC0BF00900F5CF82F46EEC0BF075
:1029000078EC0BF02CEF1DF081B803D037B0D4EF8A
:1029100014F08351630AD8A42AEF1DF08451610A90
:10292000D8A42AEF1DF085516C0AD8A42AEF1DF017
:102930008651410A42E08651440A1BE08651420A10
:10294000D8B4F0EF14F08651350AD8B4B6EF1EF0C3
:102950008651360AD8B40BEF1FF08651370AD8B427
:1029600074EF1FF08651380AD8B4D2EF1FF02AEF67
:102970001DF00798079A04017A0E826F6EEC0BF037
:102980000401780E826F6EEC0BF00401640E826F0E
:102990006EEC0BF081A8D4EF14F00401550E826F99
:1029A0006EEC0BF0D9EF14F004014C0E826F6EEC5C
:1029B0000BF078EC0BF02CEF1DF00788079A040160
:1029C0007A0E826F6EEC0BF00401410E826F6EEC9A
:1029D0000BF00401610E826F6EEC0BF0CAEF14F085
:1029E0000798078A04017A0E826F6EEC0BF00401DF
:1029F000420E826F6EEC0BF00401610E826F6EEC82
:102A00000BF0CAEF14F0010166670EEF15F067676F
:102A10000EEF15F068670EEF15F0696716D001012B
:102A20004F671AEF15F050671AEF15F051671AEF5C
:102A300015F052670AD00101000E006F000E016F01
:102A4000000E026F000E036F120011B80AD00101D0
:102A5000620E046F010E056F000E066F000E076F09
:102A600009D00101A70E046F020E056F000E066F5C
:102A7000000E076F66C100F167C101F168C102F184
:102A800069C103F1EAEC22F003BFB7EF15F0119A28
:102A9000119C0101000E046FA80E056F550E066F04
:102AA000020E076F66C100F167C101F168C102F152
:102AB00069C103F166C18AF167C18BF168C18CF10C
:102AC00069C18DF1EAEC22F003BF0BD00101000EC9
:102AD0008A6FA80E8B6F550E8C6F020E8D6F118A48
:102AE000119C0E0E51EC09F0E8CF18F10F0E51ECCD
:102AF00009F0E8CF19F1100E51EC09F0E8CF1AF106
:102B0000110E51EC09F0E8CF1BF133EC22F08AC131
:102B100004F18BC105F18CC106F18DC107F1EAEC1E
:102B200022F00782F7EC21F033EC22F00792F7EC69
:102B300021F08AC100F18BC101F18CC102F18DC17C
:102B400003F10792F7EC21F0CC0E046FE00E056F55
:102B5000870E066F050E076FEAEC22F000C118F130
:102B600001C119F102C11AF103C11BF140D013AA2E
:102B7000BCEF15F0138E139A119C119A0101800E6F
:102B8000006F1A0E016F060E026F000E036F4FC129
:102B900004F150C105F151C106F152C107F1EAEC4F
:102BA00022F003AF05D0FFEC23F0118C119A120034
:102BB0000E0E51EC09F0E8CF18F10F0E51EC09F0B0
:102BC000E8CF19F1100E51EC09F0E8CF1AF1110E0F
:102BD00051EC09F0E8CF1BF14FC100F150C101F1F8
:102BE00051C102F152C103F10782F7EC21F018C183
:102BF00000F119C101F11AC102F11BC103F1120068
:102C00000784BAC166F1BBC167F1BCC168F1BDC13F
:102C100069F14BC14FF14CC150F14DC151F14EC161
:102C200052F157C159F158C15AF107940101666731
:102C300021EF16F0676721EF16F0686721EF16F0B5
:102C4000696716D001014F672DEF16F050672DEF21
:102C500016F051672DEF16F052670AD00101000EF1
:102C6000006F000E016F000E026F000E036F120066
:102C700011B80AD00101620E046F010E056F000E3B
:102C8000066F000E076F09D00101A70E046F020E38
:102C9000056F000E066F000E076F66C100F167C179
:102CA00001F168C102F169C103F1EAEC22F003BF4E
:102CB000B9EF16F00101000E046FA80E056F550E56
:102CC000066F020E076F66C100F167C101F168C1AE
:102CD00002F169C103F166C18AF167C18BF168C174
:102CE0008CF169C18DF1EAEC22F003BF09D001013A
:102CF000000E8A6FA80E8B6F550E8C6F020E8D6FB3
:102D000033EC22F000C104F101C105F102C106F16A
:102D100003C107F1000E006FA00E016F980E026F45
:102D20007B0E036F1BEC23F000C118F101C119F1F8
:102D300002C11AF103C11BF1000E006FA00E016F5A
:102D4000980E026F7B0E036F8AC104F18BC105F1EF
:102D50008CC106F18DC107F11BEC23F018C104F101
:102D600019C105F11AC106F11BC107F1EAEC22F005
:102D700012000101A80E006F610E016F000E026FBC
:102D8000000E036F4FC104F150C105F151C106F1AE
:102D900052C107F1EAEC22F003AF0AD00101A80EFC
:102DA000006F610E016F000E026F000E036F00D006
:102DB000C80E006FAF0E016F000E026F000E036FA2
:102DC0004FC104F150C105F151C106F152C107F1E3
:102DD000FBEC22F012000784BAC166F1BBC167F1B7
:102DE000BCC168F1BDC169F14BC14FF14CC150F19B
:102DF0004DC151F14EC152F157C159F158C15AF16B
:102E00000794010166670CEF17F067670CEF17F086
:102E100068670CEF17F0696716D001014F6718EF6C
:102E200017F0506718EF17F0516718EF17F0526757
:102E30000AD00101000E006F000E016F000E026F3C
:102E4000000E036F120011B80AD00101620E046F68
:102E5000010E056F000E066F000E076F09D001010D
:102E6000A70E046F020E056F000E066F000E076FAF
:102E700066C100F167C101F168C102F169C103F1E6
:102E8000EAEC22F003BFCEEF17F00101000E046F51
:102E9000A80E056F550E066F020E076F66C100F192
:102EA00067C101F168C102F169C103F166C18AF12C
:102EB00067C18BF168C18CF169C18DF1EAEC22F038
:102EC00003BF09D00101000E8A6FA80E8B6F550E4B
:102ED0008C6F020E8D6F010E006F000E016F000EE1
:102EE000026F000E036F8AC104F18BC105F18CC122
:102EF00006F18DC107F11BEC23F018C104F119C1D3
:102F000005F11AC106F11BC107F188EC23F02AC1B3
:102F100082F40401300E82276EEC0BF02BC182F498
:102F20000401300E82276EEC0BF02CC182F40401F8
:102F3000300E82276EEC0BF02DC182F40401300EAE
:102F400082276EEC0BF02EC182F40401300E822732
:102F50006EEC0BF02FC182F40401300E82276EEC70
:102F60000BF030C182F40401300E82276EEC0BF0BE
:102F700031C182F40401300E82276EEC0BF032C1B5
:102F800082F40401300E82276EEC0BF033C182F420
:102F90000401300E82276EEC0BF012004FC100F1DD
:102FA00050C101F151C102F152C103F1010188EC9C
:102FB00023F04BEC21F012000401730E826F6EECD3
:102FC0000BF004012C0E826F6EEC0BF0078462C1D3
:102FD00066F163C167F164C168F165C169F14BC114
:102FE0004FF14CC150F14DC151F14EC152F157C199
:102FF00059F158C15AF1079402EC18F078EC0BF033
:103000002CEF1DF066C100F167C101F168C102F14A
:1030100069C103F1010188EC23F04BEC21F00401BC
:10302000630E826F6EEC0BF004012C0E826F6EEC5F
:103030000BF04FC100F150C101F151C102F152C179
:1030400003F1010188EC23F04BEC21F00401660E42
:10305000826F6EEC0BF004012C0E826F6EEC0BF0A5
:10306000FFEC23F059C100F15AC101F1010188ECD4
:1030700023F04BEC21F00401740E826F6EEC0BF028
:10308000120010820401530E826F6EEC0BF00401EB
:103090002C0E826F6EEC0BF083C32AF184C32BF1EC
:1030A00085C32CF186C32DF187C32EF188C32FF180
:1030B00089C330F18AC331F18BC332F18CC333F150
:1030C00001014DEC24F0C4EC23F000C166F101C114
:1030D00067F102C168F103C169F18EC32AF18FC3A0
:1030E0002BF190C32CF191C32DF192C32EF193C318
:1030F0002FF194C330F195C331F196C332F197C3E8
:1031000033F101014DEC24F0C4EC23F000C14FF188
:1031100001C150F102C151F103C152F140EC24F060
:1031200099C32FF19AC330F19BC331F19CC332F1A3
:103130009DC333F101014DEC24F0C4EC23F000C138
:1031400059F101C15AF102EC18F004012C0E826F02
:103150006EEC0BF0BCEF18F0118E1CA002D01CAE70
:10316000108C1BBE02D01BA4108E03018251520A88
:1031700002E10F8201D00F928251750A02E11084A0
:1031800001D010948251550A02E1108601D01096A8
:103190008351310A03E11382138402D013921394F2
:1031A00003018351660A01E056D00401660E826F66
:1031B0006EEC0BF004012C0E826F6EEC0BF000EC49
:1031C00016F088EC23F02AC182F40401300E822725
:1031D0006EEC0BF02BC182F40401300E82276EECF2
:1031E0000BF02CC182F40401300E82276EEC0BF040
:1031F0002DC182F40401300E82276EEC0BF02EC13B
:1032000082F40401300E82276EEC0BF02FC182F4A1
:103210000401300E82276EEC0BF030C182F4040101
:10322000300E82276EEC0BF031C182F40401300EB7
:1032300082276EEC0BF032C182F40401300E82273B
:103240006EEC0BF033C182F40401300E82276EEC79
:103250000BF02AEF1DF011A003D011A401D01084AF
:10326000078410B295EF19F010A479EF19F0BAC1E4
:1032700066F1BBC167F1BCC168F1BDC169F1BEC1F6
:103280006AF1BFC16BF1C0C16CF1C1C16DF1C2C1C6
:103290006EF1C3C16FF1C4C170F1C5C171F1C6C196
:1032A00072F1C7C173F1C8C174F1C9C175F1CAC166
:1032B00076F1CBC177F1CCC178F1CDC179F1CEC136
:1032C0007AF1CFC17BF1D0C17CF1D1C17DF1D2C106
:1032D0007EF1D3C17FF1D4C180F1D5C181F1D6C1D6
:1032E00082F1D7C183F1D8C184F1D9C185F181EFD1
:1032F00019F062C166F163C167F164C168F165C12B
:1033000069F1BAC186F1BBC187F1BCC188F1BDC109
:1033100089F14BC14FF14CC150F14DC151F14EC13A
:1033200052F157C159F158C15AF107940FA0B7EFA4
:1033300019F001019667A4EF19F09767A4EF19F04F
:103340009867A4EF19F09967A8EF19F0B7EF19F093
:1033500003EC15F096C104F197C105F198C106F18F
:1033600099C107F1EAEC22F003BFF0EF1CF003EC87
:1033700015F00101000E046F000E056F010E066FBF
:10338000000E076F1BEC23F011A02AD011A228D049
:1033900088EC23F0296701D005D004012D0E826F3F
:1033A0006EEC0BF030C182F40401300E82276EEC1B
:1033B0000BF031C182F40401300E82276EEC0BF069
:1033C00032C182F40401300E82276EEC0BF033C15F
:1033D00082F40401300E82276EEC0BF078EC0BF0D7
:1033E00012A8C5D012981DC01EF01E3A1E42070E2C
:1033F0001E1600011E50000AD8B483EF1AF0000117
:103400001E50010AD8B40FEF1AF000011E50020A34
:10341000D8B40DEF1AF0B5EF1AF0B5EF1AF0FFECD3
:1034200023F02EC001F12FC000F1D89001330033FA
:10343000D890013300330101630E046F000E056F55
:10344000000E066F000E076F1BEC23F0280E046FB2
:10345000000E056F000E066F000E076FEAEC22F0FB
:1034600000C131F0FFEC23F02CC001F1019F019D60
:103470002DC000F10101A40E046F000E056F000EB7
:10348000066F000E076F1BEC23F000C130F000C187
:1034900004F101C105F102C106F103C107F1640E97
:1034A000006F000E016F000E026F000E036FEAEC5A
:1034B00022F0050E046F000E056F000E066F000E61
:1034C000076F1BEC23F000C104F101C105F102C13B
:1034D00006F103C107F1FFEC23F031C000F1EAEC83
:1034E00022F000C132F032C0E8FF050F315C03E783
:1034F0008A84B5EF1AF032C0E8FF0A0F315C01E6AA
:103500008A94B5EF1AF000C124F101C125F102C17E
:1035100026F103C127F1FFEC23F005EC24F01D5048
:103520001F0BE8CF00F10101640E046F000E056F60
:10353000000E066F000E076FFBEC22F024C104F1B1
:1035400025C105F126C106F127C107F1EAEC22F0F9
:1035500003BF02D08A9401D08A8424C100F125C11E
:1035600001F126C102F127C103F12CEF1DF000C1CA
:1035700024F101C125F102C126F103C127F110AEEA
:103580004DD0109E00C108F101C109F102C10AF13C
:1035900003C10BF188EC23F030C1E2F131C1E3F15A
:1035A00032C1E4F133C1E5F108C100F109C101F113
:1035B0000AC102F10BC103F101016C0E046F070E89
:1035C000056F000E066F000E076FEAEC22F003BFD6
:1035D00004D00101550EE66F1CD008C100F109C1ED
:1035E00001F10AC102F10BC103F10101A40E046F44
:1035F000060E056F000E066F000E076FEAEC22F054
:1036000003BF04D001017F0EE66F03D00101FF0E5E
:10361000E66F1F8E11AEF0EF1CF0119E24C100F179
:1036200025C101F126C102F127C103F111A005D086
:1036300011A203D00FB0F0EF1CF010A427EF1BF085
:103640000401750E826F6EEC0BF02CEF1BF0040181
:10365000720E826F6EEC0BF004012C0E826F6EEC1A
:103660000BF088EC23F029673BEF1BF00401200EE0
:10367000826F3EEF1BF004012D0E826F6EEC0BF09B
:1036800030C182F40401300E82276EEC0BF031C1A0
:1036900082F40401300E82276EEC0BF004012E0E32
:1036A000826F6EEC0BF032C182F40401300E82277F
:1036B0006EEC0BF033C182F40401300E82276EEC05
:1036C0000BF004016D0E826F6EEC0BF004012C0EFA
:1036D000826F6EEC0BF04FC100F150C101F151C18E
:1036E00002F152C103F1010188EC23F04BEC21F00F
:1036F0000401480E826F6EEC0BF004017A0E826FAB
:103700006EEC0BF004012C0E826F6EEC0BF066C1B8
:1037100000F167C101F168C102F169C103F1010162
:1037200088EC23F04BEC21F00401630E826F6EEC09
:103730000BF004012C0E826F6EEC0BF066C100F1F1
:1037400067C101F168C102F169C103F101010A0E0B
:10375000046F000E056F000E066F000E076FFBEC86
:1037600022F0000E046F120E056F000E066F000EA1
:10377000076F1BEC23F088EC23F02AC182F40401CC
:10378000300E82276EEC0BF02BC182F40401300E58
:1037900082276EEC0BF02CC182F40401300E8227DC
:1037A0006EEC0BF02DC182F40401300E82276EEC1A
:1037B0000BF02EC182F40401300E82276EEC0BF068
:1037C0002FC182F40401300E82276EEC0BF030C161
:1037D00082F40401300E82276EEC0BF004012E0EF1
:1037E000826F6EEC0BF031C182F40401300E82273F
:1037F0006EEC0BF032C182F40401300E82276EECC5
:103800000BF033C182F40401300E82276EEC0BF012
:103810000401730E826F6EEC0BF004012C0E826FAC
:103820006EEC0BF0FFEC23F059C100F15AC101F12D
:1038300056EC1EF013A26CEF1CF004012C0E826FEC
:103840006EEC0BF086C166F187C167F188C168F143
:1038500089C169F103EC15F00101000E046F000E3F
:10386000056F010E066F000E076F1BEC23F088EC4E
:1038700023F0296741EF1CF00401200E826F44EF12
:103880001CF004012D0E826F6EEC0BF030C182F43F
:103890000401300E82276EEC0BF031C182F404017A
:1038A000300E82276EEC0BF004012E0E826F6EEC50
:1038B0000BF032C182F40401300E82276EEC0BF063
:1038C00033C182F40401300E82276EEC0BF0040148
:1038D0006D0E826F6EEC0BF003018351460A01E01E
:1038E00007D004012C0E826F6EEC0BF0EBEC16F09F
:1038F00013A49FEF1CF004012C0E826F6EEC0BF0F2
:1039000013AC8DEF1CF00401500E826F6EEC0BF0C7
:10391000139C1398139A9FEF1CF013AE9AEF1CF0B0
:103920000401460E826F6EEC0BF0139E1398139AEF
:103930009FEF1CF00401530E826F6EEC0BF038B059
:10394000B6EF1CF004012C0E826F6EEC0BF08BB006
:10395000B1EF1CF00401440E826F6EEC0BF0B6EF79
:103960001CF00401530E826F6EEC0BF00FB2BCEF33
:103970001CF00FA0EEEF1CF004012C0E826F6EEC19
:103980000BF0200EF86EF76AF66A04010900F5CF15
:1039900082F46EEC0BF00900F5CF82F46EEC0BF0C4
:1039A0000900F5CF82F46EEC0BF00900F5CF82F43C
:1039B0006EEC0BF00900F5CF82F46EEC0BF0090011
:1039C000F5CF82F46EEC0BF00900F5CF82F46EECCB
:1039D0000BF00900F5CF82F46EEC0BF078EC0BF0F5
:1039E0000F90109E12982CEF1DF00401630E826F51
:1039F0006EEC0BF004012C0E826F6EEC0BF032ECCF
:103A00001DF004012C0E826F6EEC0BF0A5EC1DF086
:103A100004012C0E826F6EEC0BF021EC1EF0040101
:103A20002C0E826F6EEC0BF00101F80E006FCD0EC4
:103A3000016F660E026F030E036F47EC1DF0040169
:103A40002C0E826F6EEC0BF037EC1EF078EC0BF066
:103A50002CEF1DF078EC0BF00301C26B0790109275
:103A60003BEF20F0D8900E0E51EC09F0E8CF00F1BA
:103A70000F0E51EC09F0E8CF01F1100E51EC09F0F6
:103A8000E8CF02F1110E51EC09F0E8CF03F101018A
:103A9000000E046F000E056F010E066F000E076F1B
:103AA0001BEC23F088EC23F02AC182F40401300ED1
:103AB00082276EEC0BF02BC182F40401300E8227BA
:103AC0006EEC0BF02CC182F40401300E82276EECF8
:103AD0000BF02DC182F40401300E82276EEC0BF046
:103AE0002EC182F40401300E82276EEC0BF02FC140
:103AF00082F40401300E82276EEC0BF030C182F4A8
:103B00000401300E82276EEC0BF031C182F4040107
:103B1000300E82276EEC0BF004012E0E826F6EECDD
:103B20000BF032C182F40401300E82276EEC0BF0F0
:103B300033C182F40401300E82276EEC0BF00401D5
:103B40006D0E826F6EEC0BF01200120E51EC09F04C
:103B5000E8CF00F1130E51EC09F0E8CF01F1140E9B
:103B600051EC09F0E8CF02F1150E51EC09F0E8CF65
:103B700003F101010A0E046F000E056F000E066FBF
:103B8000000E076FFBEC22F0000E046F120E056FA3
:103B9000000E066F000E076F1BEC23F088EC23F07D
:103BA0002AC182F40401300E82276EEC0BF02BC187
:103BB00082F40401300E82276EEC0BF02CC182F4EB
:103BC0000401300E82276EEC0BF02DC182F404014B
:103BD000300E82276EEC0BF02EC182F40401300E01
:103BE00082276EEC0BF02FC182F40401300E822785
:103BF0006EEC0BF030C182F40401300E82276EECC3
:103C00000BF004012E0E826F6EEC0BF031C182F4CA
:103C10000401300E82276EEC0BF032C182F40401F5
:103C2000300E82276EEC0BF033C182F40401300EAB
:103C300082276EEC0BF00401730E826F6EEC0BF0BA
:103C400012000A0E51EC09F0E8CF00F10B0E51EC16
:103C500009F0E8CF01F10C0E51EC09F0E8CF02F1C8
:103C60000D0E51EC09F0E8CF03F156EF1EF0060EF1
:103C700051EC09F0E8CF00F1070E51EC09F0E8CF64
:103C800001F1080E51EC09F0E8CF02F1090E51ECF8
:103C900009F0E8CF03F156EF1EF00101FFEC23F02D
:103CA000078457C100F158C101F107940101E80EE2
:103CB000046F800E056F000E066F000E076FFBECA1
:103CC00022F0000E046F040E056F000E066F000E4A
:103CD000076F1BEC23F0880E046F130E056F000EA8
:103CE000066F000E076FEAEC22F00A0E046F000E5A
:103CF000056F000E066F000E076F1BEC23F088ECBB
:103D000023F0010129678AEF1EF00401200E826F63
:103D10008DEF1EF004012D0E826F6EEC0BF030C1A2
:103D200082F40401300E82276EEC0BF031C182F474
:103D30000401300E82276EEC0BF032C182F40401D4
:103D4000300E82276EEC0BF004012E0E826F6EECAB
:103D50000BF033C182F40401300E82276EEC0BF0BD
:103D60000401430E826F6EEC0BF0120087C32AF140
:103D700088C32BF189C32CF18AC32DF18BC32EF19B
:103D80008CC32FF18DC330F18EC331F190C332F16A
:103D900091C333F10101296B4DEC24F0C4EC23F005
:103DA0000101000E046F000E056F010E066F000E7C
:103DB000076FFBEC22F00E0E0C6E00C10BF03AEC1C
:103DC00009F00F0E0C6E01C10BF03AEC09F0100E69
:103DD0000C6E02C10BF03AEC09F0110E0C6E03C12F
:103DE0000BF03AEC09F004017A0E826F6EEC0BF0E6
:103DF00004012C0E826F6EEC0BF00401350E826F05
:103E00006EEC0BF004012C0E826F6EEC0BF032ECBA
:103E10001DF0D9EF14F087C32AF188C32BF189C3B1
:103E20002CF18AC32DF18BC32EF18CC32FF18DC3DE
:103E300030F18EC331F190C332F191C333F10101FE
:103E4000296B4DEC24F0C4EC23F0880E046F130EA4
:103E5000056F000E066F000E076FEFEC22F0000EEC
:103E6000046F040E056F000E066F000E076FFBEC6B
:103E700022F00101E80E046F800E056F000E066F40
:103E8000000E076F1BEC23F00A0E0C6E00C10BF046
:103E90003AEC09F00B0E0C6E01C10BF03AEC09F094
:103EA0000C0E0C6E02C10BF03AEC09F00D0E0C6E0C
:103EB00003C10BF03AEC09F004017A0E826F6EEC4C
:103EC0000BF004012C0E826F6EEC0BF00401360E29
:103ED000826F6EEC0BF004012C0E826F6EEC0BF017
:103EE00021EC1EF0D9EF14F087C32AF188C32BF11F
:103EF00089C32CF18AC32DF18BC32EF18CC32FF112
:103F00008DC330F18FC331F190C332F191C333F1DE
:103F100001014DEC24F0C4EC23F0000E046F120EEE
:103F2000056F000E066F000E076FFBEC22F001011B
:103F30000A0E046F000E056F000E066F000E076F6D
:103F40001BEC23F0120E0C6E00C10BF03AEC09F0E2
:103F5000130E0C6E01C10BF03AEC09F0140E0C6E4E
:103F600002C10BF03AEC09F0150E0C6E03C10BF018
:103F70003AEC09F004017A0E826F6EEC0BF004014A
:103F80002C0E826F6EEC0BF00401370E826F6EEC1C
:103F90000BF004012C0E826F6EEC0BF0A5EC1DF003
:103FA000D9EF14F087C32AF188C32BF189C32CF110
:103FB0008AC32DF18BC32EF18CC32FF18DC330F149
:103FC0008EC331F190C332F191C333F10101296BFA
:103FD0004DEC24F0C4EC23F0880E046F130E056F33
:103FE000000E066F000E076FEFEC22F0000E046F5C
:103FF000040E056F000E066F000E076FFBEC22F03B
:104000000101E80E046F800E056F000E066F000EB2
:10401000076F1BEC23F0060E0C6E00C10BF03AECA0
:1040200009F0070E0C6E01C10BF03AEC09F0080E16
:104030000C6E02C10BF03AEC09F0090E0C6E03C1D4
:104040000BF03AEC09F004017A0E826F6EEC0BF083
:1040500004012C0E826F6EEC0BF00401380E826F9F
:104060006EEC0BF004012C0E826F6EEC0BF037EC53
:104070001EF0D9EF14F081B803D037B0F9EF20F07B
:1040800007A8B3EF20F00101800E006F1A0E016F38
:10409000060E026F000E036F4BC104F14CC105F117
:1040A0004DC106F14EC107F1EAEC22F003BFF9EF72
:1040B00020F045EC21F04BC100F14CC101F14DC1A4
:1040C00002F14EC103F10782F7EC21F018C104F1AF
:1040D00019C105F11AC106F11BC107F1F80E006FF5
:1040E000CD0E016F660E026F030E036FEAEC22F035
:1040F0000E0E0C6E00C10BF03AEC09F00F0E0C6EB8
:1041000001C10BF03AEC09F0100E0C6E02C10BF07D
:104110003AEC09F0110E0C6E03C10BF03AEC09F009
:1041200007840101FFEC23F057C100F158C101F1F0
:1041300007940A0E0C6E00C10BF03AEC09F00B0E5E
:104140000C6E01C10BF03AEC09F00C0E0C6E02C1C2
:104150000BF03AEC09F00D0E0C6E03C10BF03AECCB
:1041600009F0F9EF20F007AAF9EF20F00784010128
:10417000FFEC23F057C100F158C101F10794060E7E
:104180000C6E00C10BF03AEC09F0070E0C6E01C189
:104190000BF03AEC09F0080E0C6E02C10BF03AEC91
:1041A00009F0090E0C6E03C10BF03AEC09F007841C
:1041B00062C100F163C101F164C102F165C103F1A3
:1041C0000794120E0C6E00C10BF03AEC09F0130EBE
:1041D0000C6E01C10BF03AEC09F0140E0C6E02C12A
:1041E0000BF03AEC09F0150E0C6E03C10BF03AEC33
:1041F00009F00798079A0401805181197F0B0DE09F
:104200009EA8FED714EE00F081517F0BE126E75007
:10421000812B0F01AD6EFBEF20F0C0EF0AF018C14B
:1042200000F119C101F11AC102F11BC103F1000E25
:10423000046F000E056F010E066F000E076F1BEC7A
:1042400023F029A13AEF21F02051D8B43AEF21F020
:1042500018C100F119C101F11AC102F11BC103F12A
:10426000000E046F000E056F0A0E066F000E076F3A
:104270001BEC23F01200010104510013055101133E
:10428000065102130751031312000101186B196B39
:104290001A6B1B6B12002AC182F40401300E8227B4
:1042A0006EEC0BF02BC182F40401300E82276EEC11
:1042B0000BF02CC182F40401300E82276EEC0BF05F
:1042C0002DC182F40401300E82276EEC0BF02EC15A
:1042D00082F40401300E82276EEC0BF02FC182F4C1
:1042E0000401300E82276EEC0BF030C182F4040121
:1042F000300E82276EEC0BF031C182F40401300ED7
:1043000082276EEC0BF032C182F40401300E82275A
:104310006EEC0BF033C182F40401300E82276EEC98
:104320000BF012002FC182F40401300E82276EECD4
:104330000BF030C182F40401300E82276EEC0BF0DA
:1043400031C182F40401300E82276EEC0BF032C1D1
:1043500082F40401300E82276EEC0BF033C182F43C
:104360000401300E82276EEC0BF01200060E216E57
:10437000060E226E060E236E212EBCEF21F0222E99
:10438000BCEF21F0232EBCEF21F08B84020E216EB6
:10439000020E226E020E236E212ECCEF21F0222E71
:1043A000CCEF21F0232ECCEF21F08B941200FF0EE6
:1043B000226E22C023F0030E216E8B84212EDDEFAE
:1043C00021F0030E216E232EDDEF21F08B9422C00D
:1043D00023F0030E216E212EEBEF21F0030E216E50
:1043E000233EEBEF21F0222ED9EF21F01200010144
:1043F000005305E1015303E1025301E1002BBAEC44
:1044000022F0FFEC23F03951006F3A51016F420E58
:10441000046F4B0E056F000E066F000E076FFBEC6E
:1044200022F000C104F101C105F102C106F103C18E
:1044300007F118C100F119C101F11AC102F11BC144
:1044400003F107B228EF22F0EFEC22F02AEF22F07E
:10445000EAEC22F000C118F101C119F102C11AF110
:1044600003C11BF11200FFEC23F059C100F15AC146
:1044700001F1060E51EC09F0E8CF04F1070E51EC02
:1044800009F0E8CF05F1080E51EC09F0E8CF06F18C
:10449000090E51EC09F0E8CF07F1EAEC22F000C177
:1044A00024F101C125F102C126F103C127F1290E32
:1044B000046F000E056F000E066F000E076FFBEC19
:1044C00022F0EE0E046F430E056F000E066F000E15
:1044D000076FEFEC22F024C104F125C105F126C1DC
:1044E00006F127C107F1FBEC22F000C11CF101C16C
:1044F0001DF102C11EF103C11FF1120E51EC09F0B2
:10450000E8CF04F1130E51EC09F0E8CF05F1140ED9
:1045100051EC09F0E8CF06F1150E51EC09F0E8CFA7
:1045200007F10D0E006F000E016F000E026F000EFE
:10453000036FFBEC22F0180E046F000E056F000EE7
:10454000066F000E076F1BEC23F01CC104F11DC1A8
:1045500005F11EC106F11FC107F1EFEC22F06A0E52
:10456000046F2A0E056F000E066F000E076FEAEC4F
:1045700022F01200BF0EFA6E200E3A6F396BD890FF
:104580000037013702370337D8B0CBEF22F03A2F8C
:10459000C0EF22F039073A070353D8B412000331B1
:1045A000070B80093F6F03390F0B010F396F80EC48
:1045B0005FF0406F390580EC5FF0405D405F396B24
:1045C0003F33D8B0392739333FA9E0EF22F04051CB
:1045D00039271200010124EC24F0D8B012000101A7
:1045E00003510719346FE7EC23F0D89007510319F2
:1045F00034AF800F12000101346B0BEC24F0D8A013
:1046000021EC24F0D8B01200F6EC23F0FFEC23F0FC
:104610001F0E366F37EC24F00B35D8B0E7EC23F0E3
:10462000D8A00335D8B01200362F0AEF23F034B1EA
:104630000EEC24F012000101346B04510511061137
:1046400007110008D8A00BEC24F0D8A021EC24F02E
:10465000D8B01200086B096B0A6B0B6B37EC24F0B7
:104660001F0E366F37EC24F007510B5DD8A445EFD1
:1046700023F006510A5DD8A445EF23F00551095DEA
:10468000D8A445EF23F00451085DD8A058EF23F0DB
:104690000451085F0551D8A0053D095F0651D8A017
:1046A000063D0A5F0751D8A0073D0B5FD8900081F7
:1046B000362F32EF23F034B10EEC24F0346B0BECD8
:1046C00024F0D8903BEC24F007510B5DD8A475EF93
:1046D00023F006510A5DD8A475EF23F00551095D5A
:1046E000D8A475EF23F00451085DD8A084EF23F01F
:1046F000003F84EF23F0013F84EF23F0023F84EF7B
:1047000023F0032BD8B4120034B10EEC24F01200C5
:104710000101346B0BEC24F0D8B0120040EC24F013
:10472000200E366F003701370237033711EE33F0B2
:104730000A0E376FE7360A0EE75CD8B0E76EE5522F
:10474000372F9AEF23F0362F92EF23F034B12981DF
:10475000D890120040EC24F0200E366F003701375D
:104760000237033711EE33F00A0E376FE7360A0EC1
:10477000E75CD8B0E76EE552372FB6EF23F0362F5F
:10478000AEEF23F0D890120001010A0E346F200E14
:10479000366F11EE29F03451376F0A0ED890E65279
:1047A000D8B0E726E732372FCFEF23F003330233B9
:1047B00001330033362FC9EF23F0E750FF0FD8A0A5
:1047C0000335D8B0120029B10EEC24F012000451C8
:1047D00000270551D8B0053D01270651D8B0063D48
:1047E00002270751D8B0073D032712000051086F78
:1047F0000151096F02510A6F03510B6F1200010141
:10480000006B016B026B036B12000101046B056B03
:10481000066B076B12000335D8A012000351800B02
:10482000001F011F021F031F003F1EEF24F0013F66
:104830001EEF24F0023F1EEF24F0032B342B032540
:1048400012000735D8A012000751800B041F051F66
:10485000061F071F043F34EF24F0053F34EF24F018
:10486000063F34EF24F0072B342B072512000037C6
:10487000013702370337083709370A370B37120079
:104880000101296B2A6B2B6B2C6B2D6B2E6B2F6B05
:10489000306B316B326B336B120001012A510F0BFD
:1048A0002A6F2B510F0B2B6F2C510F0B2C6F2D518F
:1048B0000F0B2D6F2E510F0B2E6F2F510F0B2F6FD4
:1048C00030510F0B306F31510F0B316F32510F0BD5
:1048D000326F33510F0B336F120000C124F101C14D
:1048E00025F102C126F103C127F104C100F105C180
:1048F00001F106C102F107C103F124C104F125C190
:1049000005F126C106F127C107F112000001195077
:10491000FF0A01E11200390EC86E800EC76E280E24
:10492000C66E000EC56E1850000AD8B4C1EF24F050
:104930001850010AD8B4DAEF24F01850020AD8B49B
:10494000F3EF24F01850030AD8B40CEF25F01850F8
:10495000040AD8B434EF25F01850050AD8B44DEF46
:1049600025F01850060AD8B466EF25F01850070A4B
:10497000D8B47FEF25F01850080AD8B498EF25F086
:1049800012001950000AD8B4B7EF25F01950010AE7
:10499000D8B4BBEF25F01950020AD8B4BFEF25F008
:1049A0001950030AD8B4C3EF25F01950040AD8B43B
:1049B00036EF26F01950000AD8B4CBEF25F0195085
:1049C000010AD8B4CFEF25F01950020AD8B4D3EFBA
:1049D00025F01950030AD8B4D7EF25F01950040A6E
:1049E000D8B436EF26F01950000AD8B4DBEF25F022
:1049F0001950010AD8B4DFEF25F01950020AD8B4D3
:104A0000E3EF25F01950030AD8B4E7EF25F0195069
:104A1000040AD8B436EF26F01950000AD8B4F4EFDF
:104A200025F01950010AD8B4F8EF25F01950020A00
:104A3000D8B4FCEF25F01950030AD8B410EF26F0D3
:104A40001950040AD8B414EF26F01950050AD8B446
:104A500018EF26F01950060AD8B41CEF26F01950AA
:104A6000070AD8B41FEF26F01950000AD8B423EF74
:104A700026F01950010AD8B427EF26F01950020A7F
:104A8000D8B42BEF26F01950030AD8B42FEF26F034
:104A90001950040AD8B432EF26F01950000AD8B4DD
:104AA0003AEF26F01950010AD8B43EEF26F019501B
:104AB000020AD8B442EF26F01950030AD8B446EFE0
:104AC00026F01950040AD8B436EF26F01950000A1F
:104AD000D8B450EF26F01950010AD8B454EF26F09C
:104AE0001950020AD8B458EF26F01950030AD8B466
:104AF0005CEF26F01950040AD8B436EF26F01950AE
:104B0000000AD8B45DEF26F01950010AD8B461EF5D
:104B100026F01950020AD8B465EF26F01950030A9E
:104B2000D8B469EF26F01950040AD8B436EF26F04D
:104B30001950000AD8B46AEF26F01950010AD8B407
:104B40006EEF26F01950020AD8B472EF26F0195011
:104B5000030AD8B476EF26F01950040AD8B477EFD8
:104B600026F01950050AD8B47AEF26F012009E9666
:104B7000C580192A1200E20EC96E192A1200770E9A
:104B8000C96E192A1200020EE86E8AB4E88AE8CFCC
:104B9000C9FF192A12009E96C580192A1200E20E3A
:104BA000C96E192A1200790EC96E192A1200000E58
:104BB000C96E192A12009E96C580192A1200E20EAB
:104BC000C96E192A12007A0EC96E192A12001BBC6E
:104BD00003D0E6C1E8FF04D01B50E844E8441F09B5
:104BE000E8CFC9FF192A12009E96C580192A120023
:104BF000E20EC96E192A120011BA03D011BC01D0FD
:104C000003D0050E186E3ED00101E2670CEF26F0CE
:104C1000100EC96E0EEF26F0E2C1C9FF192A12006C
:104C2000E3C1C9FF192A1200E4C1C9FF192A120001
:104C3000E5C1C9FF192A1200C584192A1200FF0E06
:104C4000196E209E12009E96C580192A1200E20E4F
:104C5000C96E192A1200760EC96E192A1200C5846F
:104C6000192A1200FF0E196E209E1200C584182A00
:104C7000196A12009E96C580192A1200E20EC96EAA
:104C8000192A12007B0EC96E192A120011AA04D02B
:104C9000230EC96E192A12001C0EC96E192A1200A1
:104CA0009E96C580192A1200E20EC96E192A1200BA
:104CB0007C0EC96E192A1200E9D79E96C580192A62
:104CC0001200E20EC96E192A12007D0EC96E192A51
:104CD0001200DCD79E96C580192A1200E20EC96E1A
:104CE000192A12007E0EC96E192A1200CFD7C58468
:104CF000192A1200FF0E196E209E12001950FF0A89
:104D0000D8B43CEF27F0390EC86E800EC76E280E5F
:104D1000C66E000EC56E1850000AD8B497EF26F084
:104D20001850010AD8B4ABEF26F03CEF27F0195029
:104D3000000AD8B4E9EF26F01950010AD8B4EDEF13
:104D400026F01950020AD8B4F7EF26F01950030ADA
:104D5000D8B4FAEF26F01950000AD8B400EF27F0C3
:104D60001950010AD8B404EF27F01950020AD8B438
:104D70000EEF27F01950030AD8B411EF27F019509D
:104D8000040AD8B417EF27F01950050AD8B41AEF5F
:104D900027F01950060AD8B420EF27F01950070A57
:104DA000D8B423EF27F01950080AD8B429EF27F018
:104DB0001950090AD8B42CEF27F019500A0AD8B4B0
:104DC00032EF27F019500B0AD8B435EF27F03CEF3B
:104DD00027F09E96C5803BEF27F01AB004D04E0E08
:104DE000C96E3BEF27F0500EC96E3BEF27F0C5842C
:104DF0003BEF27F0182AFF0E196E12803CEF27F0C8
:104E00009E96C5803BEF27F01AB004D04F0EC96EB6
:104E10003BEF27F0510EC96E3BEF27F0C5863BEF05
:104E200027F0C9CF28F0C59AC5883BEF27F0C58683
:104E30003BEF27F0C9CF29F0C59AC5883BEF27F093
:104E4000C5863BEF27F0C9CF2AF0C59AC5883BEF4E
:104E500027F0C5863BEF27F0C9CF2BF0C58AC58860
:104E60003BEF27F0C5843BEF27F0FF0E196E12864B
:104E7000209C3CEF27F0192A120012B012D012B277
:104E800013D012B414D012A6120007B0120012965A
:104E900028C02CF029C02DF02AC02EF02BC02FF0F6
:104EA000120012901282120012921284120000015B
:104EB0001950FF0A04E11294196A7EEC26F01200E0
:104EC0001950FF0AD8B43CEF27F025EC28F0185011
:104ED000000AD8B473EF27F01850010AD8B4B1EF24
:104EE00027F03CEF27F01950000AD8B4E5EF27F07F
:104EF0001950010AD8B4EAEF27F01950020AD8B4C1
:104F0000EEEF27F01950030AD8B4F2EF27F019504A
:104F1000040AD8B4FAEF27F01950050AD8B4FDEF07
:104F200027F01950060AD8B404EF28F01950070AE0
:104F3000D8B407EF28F01950080AD8B40EEF28F0BB
:104F40001950090AD8B411EF28F019500A0AD8B438
:104F500018EF28F019500B0AD8B41BEF28F03CEFDB
:104F600027F01950000AD8B421EF28F01950010A8F
:104F7000D8B421EF28F01950020AD8B421EF28F054
:104F80001950030AD8B421EF28F01950040AD8B4F4
:104F900021EF28F01950050AD8B421EF28F0195054
:104FA000060AD8B421EF28F01950070AD8B421EF27
:104FB00028F01950080AD8B421EF28F01950090A2E
:104FC000D8B421EF28F03CEF27F09E96C596C58017
:104FD00023EF28F0520EC96E23EF28F0B40EC96EED
:104FE00023EF28F0C9CF33F0336AC586C59AC58848
:104FF00023EF28F0C58623EF28F0C9CF34F0346AB8
:10500000C59AC58823EF28F0C58623EF28F0C9CFBD
:1050100035F0356AC59AC58823EF28F0C58623EF99
:1050200028F0C9CF36F0366AC58AC58823EF28F044
:10503000C58423EF28F0FF0E196E1286209C24EF02
:1050400028F024EF28F0192A1200390EC86E800EBD
:0C505000C76E280EC66E000EC56E120062
:10BF0000E844F926000C160C2B0C3F0C520C640C68
:10BF1000760C860C960CA50CB30CC10CCF0CDC0C6B
:06BF2000E80CF40C000C1B
:00000001FF
